:020000020000FC
:100000000C949C090C942A000C942A000C942A004D
:100010000C942A000C942A000C942A000C942A00B8
:100020000C942A000C942A000C947F050C942A004E
:100030000C942A000C942A000C942A000C942A0098
:100040000C942A000C942A000C942A000C942A0088
:100050000C942A0018959198899A0895919A899AF2
:080060000895919BFBCFF7CF3F
:1002000085BAA99185BAA62B000085BAEC9185BA6A
:10021000099485BAA99185BAA62B000085BAEC91FC
:1002200075BA099485BAA99185BAA62B000075BA4A
:10023000EC9185BA099485BAA99185BAA62B0000DC
:1002400075BAEC9175BA099485BAA99175BAA62BBD
:10025000000085BAEC9185BA099485BAA99175BA5E
:10026000A62B000085BAEC9175BA099485BAA991BC
:1002700075BAA62B000075BAEC9185BA099485BAB7
:10028000A99175BAA62B000075BAEC9175BA0994BC
:1002900075BAA99185BAA62B000085BAEC9185BAEA
:1002A000099475BAA99185BAA62B000085BAEC917C
:1002B00075BA099475BAA99185BAA62B000075BACA
:1002C000EC9185BA099475BAA99185BAA62B00005C
:1002D00075BAEC9175BA099475BAA99175BAA62B3D
:1002E000000085BAEC9185BA099475BAA99175BADE
:1002F000A62B000085BAEC9175BA099475BAA9913C
:1003000075BAA62B000075BAEC9185BA099475BA36
:10031000A99175BAA62B000075BAEC9175BA09942B
:1003200095BA65E0E9D3000000000C946F0685BA29
:1003300078248724782485BAA991A62BEC91099476
:1003400085BA7424472474240000A991A62BEC914B
:10035000099485BA7524572475240000A991A62B09
:10036000EC91099485BA86246824862485BAA991DB
:06037000A62BEC9109949C
:100400000009121B242D363F48515A636C757E87B4
:1004100097A0A9B2FF93EF93043108F000E0E0E069
:10042000F4E0E00F00E0F01F0491EF91FF910895D8
:10043000101010101010101000000000000000102C
:100440001111111111111111121212121212121294
:1004500013131313131313130000060202060000F4
:100460000000060204060000000006020606000066
:10047000000006040006000000000604020600005A
:100480000000060404060000000006040606000042
:100490000000060600060000000006060206000036
:1004A000000006060406000000000606060600001E
:1004B0000000000000000000000000000303030330
:1004C000000000000C0C0C0C000000000F0F0F0FC0
:1004D00003030303000000000303030303030303F8
:1004E000030303030C0C0C0C030303030F0F0F0F88
:1004F0000C0C0C0C000000000C0C0C0C0303030390
:100500000C0C0C0C0C0C0C0C0C0C0C0C0F0F0F0F1F
:100510000F0F0F0F000000000F0F0F0F0303030357
:100520000F0F0F0F0C0C0C0C0F0F0F0F0F0F0F0FE7
:1005300000000000000000000004040404000400A7
:10054000000A0A0A00000000000A0A0E0A0E0A0A3F
:100550000004060C04060C04000A020404080A0045
:1005600000040A040A0A0600000408000000000053
:100570000004080808080400000402020202040043
:100580000000040E040E0400000004040E04040025
:100590000000000000040408000000000E0000003D
:1005A0000000000000040400000202040408080027
:1005B00000040A0A0A0A040000040C0404040E00E1
:1005C00000040A0204080E00000C020402020C00DF
:1005D00000080A0A0E020200000E080C02020C00BB
:1005E0000004080C0A0A0400000E020204040400BD
:1005F00000040A040A0A040000040A0A06020400AD
:1006000000000404000404000000040400040408C2
:1006100000000204080402000000000E000E0000AA
:100620000000080402040800000C02040400040096
:1006300000040A0E0E08060000040A0A0E0A0A0048
:10064000000C0A0C0A0A0C0000040A08080A04003C
:10065000000C0A0A0A0A0C00000E080C08080E001A
:10066000000E08080C08080000040A080A0A060020
:10067000000A0A0E0A0A0A00000E040404040E000E
:10068000000E040404040800000A0A0C0C0A0A0004
:100690000008080808080E00000A0E0E0A0A0A00E0
:1006A000000E0A0A0A0A0A0000040A0A0A0A0400DA
:1006B000000C0A0A0C08080000040A0A0A0E0600C8
:1006C000000C0A0A0C0C0A000006080402020C00C6
:1006D000000E040404040400000A0A0A0A0A0400C2
:1006E000000A0A0A0A040400000A0A0A0E0E0A0096
:1006F000000A0A04040A0A00000A0A0A04040400A0
:10070000000E020404080E0000060404040406009F
:100710000008080404020200000C040404040C0095
:100720000004040A00000000000000000000000EA9
:100730000004020000000000000000060A0A060093
:100740000008080C0A0A0C00000000060808060051
:10075000000202060A0A0600000000040A0C060055
:100760000002040E04040400000000060A06020C45
:100770000008080C0A0A0A000004000C04040E0019
:100780000004000C040404080008080A0C0C0A0009
:10079000000C040404040E000000000C0E0E0E00F9
:1007A0000000000C0A0A0A00000000040A0A040003
:1007B0000000000C0A0C0808000000060A060202ED
:1007C0000000000C0A0808000000000608060C00E3
:1007D0000004040E040402000000000A0A0A0600D5
:1007E0000000000A0A0404000000000A0A0E0E00BD
:1007F0000000000A04040A000000000A0A06020CB5
:100800000000000E04080E000002040408040402A4
:10081000000404040404040000080404020404089E
:1008200000060C00000000000000000000000000B6
:10083000000000040400000000000004040404049C
:100840000000000707000000000000070704040480
:100850000000000C0C0000000000000C0C0404045C
:100860000000000F0F0000000000000F0F04040440
:100870000404040404000000040404040404040444
:100880000404040707000000040404070704040428
:100890000404040C0C0000000404040C0C04040404
:1008A0000404040F0F0000000404040F0F040404E8
:1008B000000000000000000000000000000404042C
:1008C0000000000303000000000000010302040414
:1008D00000000008080000000000000008080404F0
:1008E0000000000F0F000000000000010B0A0404CC
:1008F00004040400000000000404040404040404CC
:1009000004040203010000000404020303020404BF
:10091000040408080000000004040808080804048F
:1009200004040A0B0100000004040A0B0B0A04046F
:100930000000000000000000000000000000000FA8
:100940000000000000000F0F00000000000F0F0F5C
:10095000000000000F0F0F0F0000000F0F0F0F0F10
:1009600000000F0F0F0F0F0F000F0F0F0F0F0F0FC4
:100970000F0F0F0F0F0F0F0F0F0F0F0F0F0F0F0096
:100980000F0F0F0F0F0F00000F0F0F0F0F000000C2
:100990000F0F0F0F000000000F0F0F0000000000EE
:1009A0000F0F0000000000000F000000000000001A
:1009B0000F0F00000000000000000F0F00000000FB
:1009C000000000000F0F00000000000000000F0FEB
:1009D00008080808080808080404040404040404B7
:1009E00002020202020202020101010101010101EF
:1009F0000F0F0808080808080F0F01010101010185
:100A00000808080808080F0F0101010101010F0F74
:100A10000F0F0E0E0C0C08080F0F07070303010140
:100A200008080C0C0E0E0F0F0101030307070F0F30
:100A30002F772F3709F40895A0E8B0E0A20F18E04F
:100A400005910E940A020C93A058BF4F1A95C1F756
:100A50000895E0E3F4E020E0EBDF23952038E1F7B0
:100A6000AFEFB0E018E000E90C93A058BF4F1A9523
:100A7000D1F708950F730D9308950D9108950F7791
:100A80000F3709F40EE20D9308950D910895FF912B
:100A9000EF91EE0FFF1F9F938F93859195910C918E
:100AA0000F3761F00591EBDF0197C9F78F919F91A7
:100AB000E0FD3196F695E795099405910197E9F7E0
:100AC000F5CF3F934F93A0E8B4E037E103E0D2DFE6
:100AD0000BE1D0DF0FE1CEDF0FE2CCDF07E1CADFB1
:100AE00044E20EE2CCDF4A95E1F70FE70D933A9529
:100AF00069F74F913F9108956A95F1F70895F09342
:100B00004C08E0934B08D0934A08C0934908B0932F
:100B10004808A09347086FB760934608000062B783
:100B2000623001F0000000000000000062B7633096
:100B300001F0000000000000000062B7643001F026
:100B4000E601F70109947F016E0162E068BF6091E0
:100B500046086FBFA0914708B0914808C091490866
:100B6000D0914A08E0914B08F0914C081895F89400
:100B7000F0934C08E0934B08D0934A08C09349087F
:100B8000B0934808A09347086FB76093460860E0A9
:100B900062BF6AE46CBF6AE063BF62E069BF0CC019
:100BA000AE98AF98A69AA79A979A8F980895AE9AFA
:100BB00067E0A2DFAE98089587996CE1879B63E4B4
:100BC000B62E6FEFA62EF3DFE7EEF5E0BCCF62E0C6
:100BD00093DF0000BA9449F000000000000000001C
:100BE0000000000000000000EECF87996DE0879BB9
:100BF0006CE0B62E6EEFA62EAF9AD9DFE1E0F6E0FC
:100C0000A2CF62E079DF0000BA9449F00000000052
:100C1000000000000000000000000000EECF8799F7
:100C200069E2879B6EE4B62E6DEFA62EAF98BFDF0C
:100C3000EBE1F6E088CF62E05FDF0000BA94D1F02C
:100C400000000000000000000000000000000000A4
:100C5000EECF0FEFA016F1F3A016F1F7089500E024
:100C6000902E95BA04B30F6304BB969A8E98959A0A
:100C70008D980895879967E1879B67E1A62EC0E864
:100C8000D4E070E0BB2493DFB0FE11C0869B11C09E
:100C900088808599892CAA966CE02EDF00000000E0
:100CA00085BAE4E5F6E04FCF95BA0C946F060000E4
:100CB000000066E021DF65E01FDF0000000060E863
:100CC000769F60E8B0E0600DB11DF1E08990799009
:100CD000499059906990A991A62BEC910994B094F0
:100CE00021F0AA9763E008DFCECF7395783029F022
:100CF000AA9761E001DF0000C5CFAA9451F000007F
:100D000000000000000000000000000000000000E3
:100D1000B8CF0000000000004FCF373160F415302D
:100D200050F4A0E8B4E02AE2329FA00DB11DA10F5B
:100D300020E0B21F9FCE08953731E8F71530D8F77D
:100D4000A0E8B4E02AE2329FA00DB11DA10F20E07F
:100D5000B21F93CE373178F7443268F7A5E8B4E094
:100D60002AE2329FA00DB11DA40F20E0B21F87CE52
:100D7000373108F74432F8F6A5E8B4E02AE2329FAA
:100D8000A00DB11DA40F20E0B21F81CEF1DF240021
:100D90002020202020202020202020202020202053
:100DA0002020202020202020202020202020202043
:100DB0002020202033950895DBDF200020212223EE
:100DC0002425262728292A2B2C2D2E2F303132336B
:100DD0003435363738393A3B3C3D3E3F3395C8DFF2
:100DE0002000404142434445464748494A4B4C4D08
:100DF0004E4F505152535455565758595A5B5C5D9B
:100E00005E5F3395B5DF200060616263646566678D
:100E100068696A6B6C6D6E6F7071727374757677DA
:100E200078797A7B7C7D7E2033950895AFDFAEDFC5
:100E3000ADDF33504E5FC0DF4250089500E010E058
:100E40006CDFA4CF10E069DF00E011E066DF3395CE
:100E5000089500E3F7DF0CE3F5DF0CE0F3DF0FE0CC
:100E6000F1DF03E0EFDF03E3EDDF3650089580DFCD
:100E700013002D275F5F602D2E5F5F2E2D275F5F94
:100E8000602D2E5F5F0033950895F1DFF0DFEFDF17
:100E9000EEDFEDDFECDF08950FE15CDF33950895C1
:100EA000FBDFFADFF9DFF8DFF7DFF6DF089560DF59
:100EB000100010131313131313131313131313131B
:100EC0001310339555DF100010111210101012116D
:100ED000101111101310121033954ADF1000101961
:100EE000101110171217121515151015151033952E
:100EF0003FDF100010101A1A1A15101510141615CD
:100F000015151D10339534DF1000101C101410142B
:100F10001010181018101C141410339529DF10002D
:100F2000101C1C1C1C1C1C1C1C1C1C1C1C1C1C1019
:100F300033950895AADF36504D5EB2DF36504395A3
:100F4000B6DF4451089514DF240041546D65676194
:100F50003332207543202B20536F6674564741204F
:100F60003D203430306C696E65203730487A3395D7
:100F7000FFDE240031382E3433324D487A2C2033B2
:100F8000636C6B2F70782C203470782F63686172DB
:100F90002C203430636861723395EADE2400206EC1
:100FA00065696C2E6672616E6B6C696E2E63682F5C
:100FB00050726F6A656374732F536F66745647413E
:100FC0002F20339508950F9300E010E0A6DE0F91D7
:100FD0000F9311E0A2DE0F910F930A7212E09DDED3
:100FE0000F910F930A6213E098DE0F91057114E0E0
:100FF00094DE3395089503E0E6DF0CE0E4DF0FE0D4
:10100000E2DF00E3E0DF03E3DEDF0CE3DCDF0FE33E
:10101000DADF37500895ACDE24006E6F7200696E1F
:1010200076006E6F01756C696E016E6F02666731D6
:10103000026E6F03666732036E6F04626733339527
:101040000895E9DFE8DFE7DFE6DFE5DFE4DFE3DFA0
:10105000E2DF089510E070DE005F5FDE0895949A8D
:101060008C9884990895052F0F7341F43F9330E0D5
:10107000F1DF3395EFDF3395EDDF3F9108953F9337
:101080004F933EE040E082DE3150939A8B988399F3
:1010900010C040914D08052F0F7031F44395443234
:1010A00008F040E040934D0863DE04005F405F2F8E
:1010B00033954F913F9108955BDE08001F1010108B
:1010C0001010101F33950895F7DFF6DFF5DFF4DF1A
:1010D000F3DFF2DF089500000000000000000000D0
:1010E0000000000000000000010C00030E000202DE
:1010F00000040100040100080008080008080008B6
:10110000080008080008080008080008080008048B
:101110000100040100020200030E00010C000000A7
:1011200000000000000000000000000000000000BF
:1011300011FBC6F410FB6EF445FB04F906954795C8
:1011400045FB04F90695479545FB04F90695479537
:101150000FC046FB04F90695479546FB04F9069532
:10116000479506C010FB26F447FB04F90695479502
:101170000895A0E8B0E0A20F3F934F9338E040E01D
:1011800005910E9498080E940A020D9305910E9401
:1011900098080E940A020D9305910E9498080E94E7
:1011A0000A020D93A350A058BF4F3A9541F74F91B3
:1011B0003F910895E8EEF0E126E0029FE019F10981
:1011C00027E0D7DF2D5F2031E1F70895D1DD03005F
:1011D000070809003395CCDD03000A0B0C0033959A
:1011E000C7DD03000D0E0F00339508953F934F9315
:1011F00034E040E04ADE3650929A8A98829924C0C0
:101200004CE062DF36504395052F0695102F16955A
:101210001C5F0F711F71202F24FD0FE124FD021BA5
:10122000212F24FD1FE124FD121B0F931F93037038
:1012300013700E94DA081F910F9106950695300FE2
:1012400016951695410FC2DF4F913F9108953F9338
:101250004F933BE040E077DE3350919A8998819933
:1012600011C050FD0FC054FD0DC040914E08052F18
:101270000F7331F44395443208F040E040934E0838
:101280000FE168DD4F913F910895000E0A0A0A0AA6
:101290000E00000C040404040E00000E02020E08EE
:1012A0000E00000E020E02020E00000A0A0A0E02D2
:1012B0000200000E080E02020E00000E080E0A0ABE
:1012C0000E00000E020202020200000E0A0E0A0ABE
:1012D0000E00000E0A0A0E020E0020E3A9DB239581
:1012E0002A33E1F70895E0EBF5E00E946D09909A4A
:1012F0008898809907C0052F007221F4EAE8F2E18E
:101300000E946D09089530E040E090DD97DDA1DD99
:1013100011DE94DD18DE92DD6EDE93DE8FDD50E0AF
:1013200050934D0850934E0894DC539598DEA7DEF9
:101330005DDF8DDFD8DFF8CFAFE7B0E0ADBFBEBF78
:0E134000789487DBBEDB2CDC8ADC11DCDCCF92
:00000001FF
